:10000000F89411240FEF0DBF00E10EBFA0E0B1E0A6
:10001000C8EFD1E0CA1BDB0B2196EAECF9E021978F
:1000200019F005900D92FBCFA8EFB1E0C4E0D2E04B
:10003000CA1BDB0B2196219711F01D92FCCF02D039
:100040000C9402F0AF92BF92CF92DF92EF92FF92A8
:100050000F931F93CF93DF93CDB7DEB765970FB69E
:10006000F894DEBF0FBECDBF80E091E00E94D203C6
:1000700085E291E00E94D2038AE491E00E94D203DB
:1000800083E791E00E94D2036CE971E080E090E0A8
:100090000E94CC026DE971E081E090E00E94CC0208
:1000A00080E090E0FE01E80FF91F118201968F3089
:1000B0009105C0F32FEFE22EF22E670100E010E071
:1000C0005801AE01405F5F4FBE016E5E7F4FCE01B3
:1000D00044960E94E30089EA91E00E94D2036AE01C
:1000E00070E08C899D890E94460180EB91E00E941E
:1000F000D203EA89FB89EE0FFF1FEE0FFF1FEE53BD
:10010000FE4F88899989E80FF91F80810E94B0030A
:1001100083ED91E00E94D2034A895B89FA01EE0FD8
:10012000FF1FEE0FFF1FEA52FE4F88899989E80FE3
:10013000F91F2081233279F4AA24BB2401501040F6
:1001400017FD07C0FE01E00FF11F80E2818301501F
:10015000104020E21AC0203229F4AA24BB24015006
:10016000104013C04C155D0571F48E159F0559F4B0
:100170008C899D898436910534F40150104008948F
:10018000A11CB11C02C0AA24BB24203251F0FE01E4
:10019000E00FF11FC50163E070E00E94B004280F7A
:1001A0002183BE016F5F7F4F80E090E00E94CC0210
:1001B000CA88DB88E888F9880F5F1F4F0E30110569
:1001C0000CF47FCF61CFAF92BF92CF92DF92EF92CC
:1001D000FF920F931F93CF93DF935C017B016A0122
:1001E0008FE084BB1ABA00E010E0C0E0D0E08FE0FE
:1001F0008BBB21E030E0C9010C2E02C0880F991F93
:100200000A94E2F780958F7085BB60E070E0C901C9
:100210000E949C0189B3282F33272F7030700F5F05
:100220001F4F40E050E0C901042E02C0959587950C
:100230000A94E2F780FF05C04F5F5F4F44305105DD
:1002400094F34430510589F089B399278F709070E9
:1002500082179307C9F3F701C083D183F601408366
:100260005183F5010083118306C02196C430D10566
:100270000CF4BDCFBACFDF91CF911F910F91FF90BA
:10028000EF90DF90CF90BF90AF900895EF92FF92E4
:100290000F931F93CF93DF937C018B016131710525
:1002A00010F000E110E0C701B8010E949C04EB01CE
:1002B000672B69F0B801CE010E944601C09FC001C2
:1002C000C19F900DD09F900D1124E81AF90A87EE76
:1002D00091E0E80EF91EF70180810E94B003DF91E2
:1002E000CF911F910F91FF90EF900895A091F80189
:1002F000B091F901AB2BA9F4109290006FE069B9AD
:1003000052E05BB948E14AB936E0309395008F9AE4
:1003100097988E98969A21E030E03093F9012093D7
:10032000F8015F9904C097985F9BFECF979A8CB1B4
:10033000992787FD909508952F923F924F925F9253
:100340006F927F928F929F92AF92BF92CF92DF92E5
:10035000EF92FF920F931F93CF93DF93CDB7DEB74A
:100360002A970FB6F894DEBF0FBECDBF8D839E8354
:100370006F8378871FBC01E00EBD10927A004CB4E9
:1003800049823DB43A8229803A80609000027090A0
:100390000102261837083694279436942794369409
:1003A00027944090FE015090FF01420C531C509244
:1003B000FF014092FE014101AA24BB24D501C401E2
:1003C000E3E0880F991FAA1FBB1FEA95D1F7881990
:1003D0009909AA09BB09680E791EC501B40120E478
:1003E00030EB45E050E00E947D048090FA0190904F
:1003F000FB01A090FC01B090FD01860E971EA81E87
:10040000B91EC501B40120E432E44FE050E00E947F
:10041000C304DA01C90129833A83620E731E709204
:10042000010260920002AA27BB27BC01CD0120E493
:1004300032E44FE050E00E947D04861A970AA80A31
:10044000B90A8092FA019092FB01A092FC01B0924D
:10045000FD0112011FBC11E01EBD10927A00FCB418
:10046000FB82DDB4DC822B813C812619370936956D
:10047000279536952795369527957201E20EF31E3E
:100480002701E986FA8644275527DA01C90163E086
:10049000880F991FAA1FBB1F6A95D1F7821B930B68
:1004A000A40BB50B8301080F191FCA01B90120E481
:1004B00030EB45E050E00E947D046B017C01C80CEC
:1004C000D91CEA1CFB1CC701B60120E432E44FE052
:1004D00050E00E94C304DA01C9012B833C83020F60
:1004E000131F3801AA27BB27BC01CD0120E432E449
:1004F0004FE050E00E947D04C61AD70AE80AF90AC4
:1005000046015701C201821993094D815E81452B35
:1005100071F033E0883E930708F49CCF6D817E81B3
:10052000615070406D837E83280E391E93CF2F81DA
:1005300038858217930728F4281B390B2F833887B7
:10054000F3CFC092FA01D092FB01E092FC01F0924D
:10055000FD01109301020093000269847A84709275
:10056000FF016092FE012A960FB6F894DEBF0FBE1F
:10057000CDBFDF91CF911F910F91FF90EF90DF9052
:10058000CF90BF90AF909F908F907F906F905F9033
:100590004F903F902F9008950F931F93CF93DF9329
:1005A000EC018B01A0910202B0910302AB2B61F12F
:1005B000CD2B41F160EC80E090E00E945203C0E05E
:1005C000D0E0D8016C91662381F48E012196003130
:1005D00011051CF560E281E090E00E945203AE013B
:1005E000219640315105B4F318C00F5F1F4F81E0D1
:1005F00090E00E9452032196D8013C91632F33234F
:10060000A1F7E3CF60E8D7CF0E94120321E030E0EA
:100610003093030220930202CBCFDF91CF911F9141
:100620000F9108952FEF27BB21B32F6021BB60E00E
:1006300070E08FE090E00E949C0160E380E090E039
:100640000E94650360E070E085E090E00E949C01FC
:1006500060E380E090E00E94650364E670E080E083
:1006600090E00E949C0160E380E090E00E946503BE
:1006700068E380E090E00E94520368E080E090E050
:100680000E94520361E080E090E00E94520363E028
:1006900080E090E00E9452036DE080E090E00E94D4
:1006A000520308951F93CF93DF93EC01162F80E040
:1006B00090E00E947D0387FDFACF612FCE010E945A
:1006C0006503DF91CF911F9108952FEF27BB892BF1
:1006D00011F4939801C0939A9198929A68BB61E043
:1006E00070E080E090E00E949C01929861E070E0F0
:1006F00080E090E00E949C0108951F9317BA892B17
:1007000011F4939801C0939A919A929A61E070E0E3
:1007100080E090E00E949C0116B3929861E070E046
:1007200080E090E00E949C01812F992787FD9095A1
:100730001F910895109290005FE059B942E04BB9C3
:1007400038E13AB926E0209395008F9A97988E98D1
:10075000969A21E030E03093F9012093F801089552
:10076000282FA091F801B091F901AB2BA9F41092B8
:1007700090007FE079B962E06BB958E15AB936E090
:10078000309395008F9A97988E98969A41E050E012
:100790005093F9014093F8018699FECF5D9BFCCF01
:1007A0002CB90895CF93DF93EC018881882331F031
:1007B00021960E94B00388818823D1F7DF91CF91E1
:1007C00008956F927F928F929F92AF92BF92CF9235
:1007D000DF92EF92FF920F931F93CF93DF93CDB7EA
:1007E000DEB722970FB6F894DEBF0FBECDBF1FBC99
:1007F00001E00EBD10927A007CB479826DB46A82F9
:1008000029813A81809000029090010228193909CB
:100810003695279536952795369527956090FE0154
:100820007090FF01620E731E7092FF016092FE01D4
:100830006901EE24FF24D701C60113E0880F991F38
:10084000AA1FBB1F1A95D1F78C199D09AE09BF09C4
:10085000880E991EC701B60120E430EB45E050E058
:100860000E947D04E090FA01F090FB010091FC01F0
:100870001091FD01E60EF71E081F191FA0E4AA2E15
:10088000A2E4BA2EAFE0CA2ED12CC801B701A6014E
:1008900095010E94C304DA01C901820E931E909251
:1008A000010280920002AA27BB27BC01CD01A6014C
:1008B00095010E947D04E61AF70A080B190BE092D5
:1008C000FA01F092FB010093FC011093FD01C301BA
:1008D00022960FB6F894DEBF0FBECDBFDF91CF9149
:1008E0001F910F91FF90EF90DF90CF90BF90AF904E
:1008F0009F908F907F906F900895629FD001739F1B
:10090000F001829FE00DF11D649FE00DF11D929FAB
:10091000F00D839FF00D749FF00D659FF00D9927EA
:10092000729FB00DE11DF91F639FB00DE11DF91F0E
:10093000BD01CF0111240895AA1BBB1B51E107C0C3
:10094000AA1FBB1FA617B70710F0A61BB70B881F5F
:10095000991F5A95A9F780959095BC01CD010895EE
:1009600097FB092E07260AD077FD04D0E5DF06D0D5
:1009700000201AF4709561957F4F0895F6F79095D1
:1009800081959F4F0895A1E21A2EAA1BBB1BFD0162
:100990000DC0AA1FBB1FEE1FFF1FA217B307E4075E
:1009A000F50720F0A21BB30BE40BF50B661F771FB6
:1009B000881F991F1A9469F7609570958095909596
:0A09C0009B01AC01BD01CF010895B9
:1009CA004C696E6B205042302D50423720746F2094
:1009DA004C43442044302D4437202838207769720C
:1009EA006573290A004C696E6B205044302D5044BF
:1009FA003320746F204C43442042452D5253202803
:100A0A0034207769726573290A004C696E6B20502D
:100A1A0043302D50433320746F204B6579706164E5
:100A2A002052302E2E523320283420776972657373
:100A3A00290A004C696E6B205041302D50413320F9
:100A4A00746F204B65797061642043302E2E4333D6
:100A5A00202834207769726573290A000054657862
:100A6A0074696E67204C6162004166746572200089
:100A7A006D7320796F7520747970656420613A20EE
:100A8A0027003132334134353642373839432A3038
:100A9A00234400270A0020414420474A4D2050544D
:100AAA00572020202344003031323334353637384A
:080ABA00394142434445460066
:00000001FF
